:1000000012C02AC02AC028C043C026C025C024C0B0
:1000100023C022C021C020C01FC01EC01DC01CC0E4
:100020001BC01AC019C011241FBECFEDCDBF10E0F8
:10003000A0E6B0E0E4E4F1E002C005900D92A23643
:10004000B107D9F710E0A2E6B0E001C01D92A436D6
:10005000B107E1F75AD074C0D3CF1F920F920FB6F9
:100060000F9211248F931DBC1CBC86B38095809386
:100070006200109263001092600089E08EBD929A37
:1000800096981BBE8F910F900FBE0F901F901895E2
:100090001F920F920FB60F9211248F939F939091FE
:1000A00063009F5F9093630080916000823051F401
:1000B0009F3F21F5929880E88BBF1092600088E006
:1000C0008EBD1CC0813069F49233C1F488E08EBDCE
:1000D00088EE88BF80EE8ABF80E88BBF10926000F8
:1000E0000DC0882359F480916200981738F09298D7
:1000F000969A1092630081E0809360009F918F91A7
:100100000F900FBE0F901F90189504D0789489E03F
:100110008EBDFFCF17BA8FEF88BB8FE782BB84E419
:1001200081BB8BE085BF88E08EBD80E489BF1DBCAC
:100130001CBC85E28BBD8EE08ABD89E481BF089539
:04014000F894FFCF61
:020144000200B7
:00000001FF
